:0400000070EF05F0A8
:1000080000C016F001C015F0E1CF17F0E2CF18F0EC
:100018009DAA77D09EAA75D0AECF60F0ABA40ED0C3
:10002800AB9E010E1D24006E000E1E20016E00C046
:100038001DF001C01EF0AB8E0001606BABA20ED0AC
:100048000001AB98AB88010E5824006E000E5920B1
:10005800016E00C058F001C059F0606B0001000E3D
:10006800B61902E1010EB51918E1F90E0101492589
:10007800E16E000E4A21E26EE66A010E0001F76F9A
:10008800000EF86F49C1F5F04AC1F6F00101496B5D
:100098004A6BAECF60F09D9A17D00101F90E492541
:1000A800E16E000E4A21E26E60C0E6FF010E4925AE
:1000B800006E000E4A21016E00C049F101C04AF1EC
:1000C80049C1F5F04AC1F6F0800E006E800E4A195B
:1000D800005C02E14951500814E2020E0001F76F7A
:1000E800000EF86F9D9A020E0101495D006E000E28
:1000F8004A59016EF90E0024E16E000E0120E26EED
:10010800E66A9DA01FD09EA01DD0010E0001F35DE0
:10011800006E000EF459016E00C0F3F001C0F4F057
:10012800000EF45D02E1010EF35D07E2F36BF46B80
:10013800010EB56F000EB66F9D903C0ECF6EB00EDF
:10014800CE6E9E9016C000F015C001F017C0E1FFFA
:0601580018C0E2FF1100D7
:10015E000101571D206E080E216E8994CBEC00F024
:10016E002032D8B0BEEF00F08984BFEF00F0899442
:10017E00CBEC00F0212EB7EF00F08984CBEC00F031
:10018E00CBEC00F0D8EF00F01C0E226E0000000049
:10019E0000000000222ECDEF00F000000000000055
:0601AE0012000000120027
:1001B40056C100F001015607005228E052C1E9FF80
:1001C40053C1EAFFEE50000A0CE052C1E9FF53C1EB
:1001D400EAFF54C1D9FF55C1DAFFEE50DE1801E140
:1001E4000FD052C1E9FF53C1EAFF54C1D9FF55C131
:1001F400DAFFDE50EE5C006E016A000E015A08D090
:100204000101524B532B544B552BD2D7006A016A30
:020214001200D6
:10021600086A096A100E0C6E013408360936045055
:10022600085E0550D8A0053C095ED8B007D004503A
:1002360008260550D8B0053C0926D8900036013668
:060246000C2EEAD71200A5
:10024C0052C102F053C103F002C000F003C001F030
:10025C00024A032A00C0E9FF01C0EAFFEE5201E0A6
:10026C00F3D701015251025C006E53510358016ED9
:0A027C00010E005E000E015A120090
:10028600086A080E0C6E003408360450085ED8B0B2
:0E02960002D00826D89000360C2EF5D71200A4
:1002A40052C1E9FF53C1EAFFEE500101541905E1BF
:1002B40052C100F053C101F010D052C100F053C13B
:1002C40001F0524B532B00C0E9FF01C0EAFFEECF0F
:0C02D40000F00052E5E1006A016A12002F
:1002E0000101546B556B52C103F053C104F052C16C
:1002F00005F053C106F003C0E9FF04C0EAFFEE5069
:10030000200A04E15451551101E110D0010E546F3F
:10031000000E556F03C0E9FF04C0EAFF05C0E1FF0E
:1003200006C0E2FFEECFE6FF054A062A03C001F051
:1003300004C002F0034A042A01C0E9FF02C0EAFF38
:10034000EE50000AD8E152C100F053C101F0120092
:0E035000ACB202D00000FCD752C1ADFF1200CB
:0C035E00420E0D6E0D2EFED700001200A6
:0A036A000000000000000000120077
:0E037400670E0D6E0D2EFED700000000120069
:1003820052C1F6FF53C1F7FF54C1F8FF0900F5CF80
:1003920000F0005210E052C1F6FF53C1F7FF54C102
:1003A200F8FF0900F5CF57F1D9DE010E5227000EF2
:0803B20053235423E5D7120088
:1003BA000B6A0A6A096A00500402F4CF09F0F3CF03
:1003CA0008F001500502F4CF0BF0F3CF0AF0005009
:1003DA000502F3500926F4500A22E86A0B2201505A
:1003EA000402F3500926F4500A22E86A0B2208C0D4
:1003FA0000F009C001F00AC002F00BC003F01200BD
:10040A00030E0C6E950E0D6E0D2EFED70C2EFCD71C
:02041A001200CE
:10041C00FF0E0001DB6FFF0EDC6F000EDD6F000EB8
:10042C00DE6FFF0EBF6FFF0EC06F000EC16F000EB0
:10043C00C26FFF0EC36FFF0EC46F000EC56F000EB0
:10044C00C66FFF0EB76FFF0EB86FFF0EB96FFF0EC2
:10045C00BA6FFF0EBB6FFF0EBC6FFF0EBD6FFF0EB2
:10046C00BE6FFF0EC76FFF0EC86F000EC96F000E78
:10047C00CA6F949894968B988B9694889486C79E02
:08048C00C79C380EC66E120079
:100494004BC1F6FF4CC1F7FF4DC1F8FF0900F5CF82
:1004A40000F0005211E04BC1F6FF4CC1F7FF4DC103
:1004B400F8FF0900F5CF52F149DF010E01014B2786
:0A04C400000E4C234D23E4D7120074
:1004CE0001014E6B4CAF0BD0010E4E6F2D0E000185
:1004DE00636F01014B1F4C1F4B4B4C2B04D04E6BCB
:1004EE00200E0001636F4BC100F04CC101F00132D0
:1004FE000032019E01320032019E01320032019E15
:10050E0001320032019E00C04DF10A0E046EB4DEBF
:10051E000A0E046EB1DE08C000F0300E0024016E2B
:10052E0001C064F00150300A03E10001200E646F37
:10053E0000010A0E046E4DC100F09EDE08C000F0F0
:10054E00300E0024656F0F0E01014B15006E4CC16D
:10055E0001F0000E0116710E046E020E056E26DFFE
:10056E0000C04FF101C050F12E0E0001666FE80E73
:10057E00046E030E056E4FC100F050C101F044DE53
:10058E00300E0024676F640E046E000E056E4FC1B0
:10059E0000F050C101F038DE0A0E046E000E056E3A
:1005AE0033DE08C000F009C001F0300E0024686F81
:1005BE00696B6A6B6B6B640E0101526F000E536FA9
:0805CE0088DE4EC100F01200AE
:1005D6000D0E0101576FC0DD0A0E576FBDDD12000B
:1005E6004DC101F0010E006E015004E0003600908E
:1005F600FF0FFBD700C051F1001E00C050F14BC1E8
:10060600E9FF4CC1EAFF0050EF16120EE926010180
:100616004F6B4F51070815E34FC100F04EC101F073
:10062600005004E00132019EFF0FFBD75051EF1638
:1006360001A002D05151EF129ADE5151EF124F2B09
:0C064600E8D7120EE95E88DE87DE1200A5
:10065200300ECD6E9E903C0ECF6EB00ECE6E4BC164
:10066200F3F04CC1F4F00001B56BB66B9E909D9017
:06067200CD809D80120006
:10067800000E01014C1902E1000E4B1934E04BC188
:10068800E9FF4CC1EAFFEE522EE04DC152F14EC1D6
:1006980053F1D8DD00C056F14BC152F14CC153F1B2
:1006A8004DC154F14EC155F181DD000E011802E132
:1006B800000E001805E14BC100F04CC101F015D047
:1006C800010E01014B25526F000E4C21536F4DC195
:1006D800E9FF4EC1EAFFEECF54F1E0DD00C04BF177
:0C06E80001C04CF1C5D7006A016A120085
:1006F40001014E6B4BC1E9FF4CC1EAFFEECF4DF156
:100704004D51000A0EE04DC152F120DE01014E2B85
:100714004E514B25E96E000E4C21EA6EEECF4DF1A1
:04072400EFD71200F9
:1007280001014F6B050E4F5D0AE24F514D25E16EF9
:10073800000E4E21E26E200EE66E4F2BF3D74F517E
:100748004D25E16E000E4E21E26EE66A4F074F51CD
:100758004D25506F000E4E21516F0A0E046E000E8B
:10076800056E4BC100F04CC101F051DD08C000F02E
:1007780009C001F0300E002650C1E1FF51C1E2FF6F
:1007880000C0E6FF0A0E046E000E056E4BC100F0B5
:100798004CC101F03CDD00C04BF101C04CF1000E32
:1007A800011802E1000E001801E102D04F07CFD76F
:0207B80012002D
:1007BA004DC101F0010E006E015004E000360090B8
:1007CA00FF0FFBD700C04FF1001E4BC1E9FF4CC120
:1007DA00EAFF0050EF16120EE9260050EF1610DE5F
:1007EA0001014F51EF12120EE95EBFDD4F51EF14B6
:1007FA004E6F4E51000A000ED8A4010E4E6F00DE55
:06080A004EC100F01200D7
:10081000016A026A800E0218006E800E000A005CF7
:1008200002E14F0E015C0AE2F90E0124E16E000EB6
:100830000220E26EE66A014A022AECD7AECF60F0EF
:100840000001F96B606B0101496B4A6B0001F56BAC
:0A085000F66BF76BF86B9D8A12003F
:10085A004BC1E9FF4CC1EAFFEE5000080AE24BC166
:10086A00E9FF4CC1EAFFEECF57F174DC4B4B4C2B3E
:04087A00EFD71200A2
:10087E000D0E0101526F65DD0A0E0101526F61DD31
:02088E00120056
:100890000001B36BB46B800EB419006E800E005C67
:1008A00002E10A0EB35D27E2030E006E000E016E38
:1008B000B3C004F0B4C005F080DD2E0E0024E96E54
:1008C000000E0120EA6EEECF52F1EECF53F1EECFE3
:1008D00054F157DD070E0B6E170E0C6E6A0E0D6E7F
:1008E0000D2EFED70C2EFCD70B2EFAD700000001E0
:0808F000B34BB42BD0D712006A
:1008F800806A0F01386B3881230E926E929889882E
:100908009296898692948984396BFF0E816E8F0E38
:10091800936EF19E3A6B826AFF0E946E949C949249
:0809280094908B80606A1200BC
:100930000900F5CFE6FF0006FBE10106F9E1120030
:100940004DC101F0010E006E015004E00036009030
:10095000FF0FFBD700C051F1001C0101506F4F6B1E
:100960004BC1E9FF4CC1EAFF4E6B4E51070820E333
:100970005051EF16120EE9265051EF16F6DC515188
:10098000EF12F3DC120EE95E5151EF14006E0CE031
:100990004EC101F0010E006E015004E000360090DF
:1009A000FF0FFBD700504F13DADCD9DC4E2BDDD71D
:0609B0004FC100F012002F
:1009B6004DC1F6FF4EC1F7FF4FC1F8FF0900F5CF55
:1009C60000F0005218E04DC1F6FF4EC1F7FF4FC1CF
:1009D600F8FF0900F5CF00F04BC1E1FF4CC1E2FF83
:1009E60000C0E6FF01014B4B4C2B010E4D27000EBC
:1009F6004E234F23DDD74BC1E1FF4CC1E2FFE66A30
:020A06001200DC
:100A0800500E0001D36F030ED46F520ED56F010E36
:100A1800D66FFF0ED76FFF0ED86F000ED96F000E7E
:100A2800DA6FFF0ECB6FFF0ECC6F000ECD6F000E8E
:100A3800CE6FFF0ECF6FFF0ED06F000ED16F000E7E
:100A4800D26FAC8A900EAB6E948E949C9EAA03D003
:080A5800AECF00F0FBD7120045
:100A60004BC100F00032009E0032009E0032009E1A
:100A70000032009ED30E0024F66E170EF76E000EA5
:100A8000F722000EF86E000EF8220900F5CF00F0F4
:100A90004CC1E1FF4DC1E2FF00C0E6FF010E0101C4
:100AA0004C25E16E000E4D21E26E0F0E4B15006ECF
:100AB000D30E0024F66E170EF76E000EF722000E0E
:100AC000F86E000EF8220900F5CF00F000C0E6FF36
:100AD000020E4C25E16E000E4D21E26EE66A120018
:100AE00045EC0CF09B6A720ED36E9B9CD26AD3B419
:100AF00001D0FDD701DF206A216A226A236A6BDDFB
:100B00000001B36BB46B800EB419006E800E005CF4
:100B100002E1040EB35D21E289968988070E0B6E0F
:100B2000170E0C6E6A0E0D6E0D2EFED70C2EFCD716
:100B30000B2EFAD7000089868998070E0B6E170EC8
:100B40000C6E6A0E0D6E0D2EFED70C2EFCD70B2EE2
:100B5000FAD70000B34BB42BD6D789868998566A4A
:100B6000576A586A596A1D6A1E6A546A556AAB6A9E
:100B7000AB88AB8EAB8A5A6A5B6A7082606B89986D
:100B8000630E616F000E626FB886010EB06EA00E2C
:100B9000AF6EAC8439DF050E0B6E0F0E0C6EF10ECE
:100BA0000D6E0D2EFED70C2EFCD70B2EFAD770DE55
:100BB000899411DDAF0E526F170E536F000E546FF4
:100BC000C1EC01F00A0EC86E29DC0B0E0B6E260E6E
:100BD0000C6E5D0E0D6E0D2EFED70C2EFCD70B2E5F
:100BE000FAD7000000003A0E0101526F170E536F42
:100BF000000E546FC1EC01F0EEDC9D809D8AF28CFA
:100C0000F28E860E526F160E536F000E546FC1ECAB
:100C100001F08B900B0E0B6E260E0C6E5D0E0D6EA2
:100C20000D2EFED70C2EFCD70B2EFAD7000000009D
:100C3000290E01014B6F180E4C6F000E4D6F2ADC10
:100C4000030E0B6E080E0C6E770E0D6E0D2EFED77A
:100C50000C2EFCD70B2EFAD7590E01014B6F180E34
:100C60004C6F000E4D6F16DC030E0B6E080E0C6EF3
:100C7000770E0D6E0D2EFED70C2EFCD70B2EFAD74D
:100C8000240E0101526F150E536F000E546FC1EC0C
:100C900001F0720E0101526F180E536F000E546F67
:100CA000C1EC01F0B5DD140E01014B6F000E4C6F6D
:100CB000D0DC6A0E01014B6F180E4C6F000E4D6FA9
:100CC0004AEC02F0030E0B6E080E0C6E770E0D6EE2
:100CD0000D2EFED70C2EFCD70B2EFAD7000E0001DE
:100CE000B61902E1000EB51907E1000EF81902E18C
:100CF000000EF71901E1F2D7B56BB66B000EF819CB
:100D000002E1010EF7190AE0800E006E800EF6195E
:100D1000005C02E1F551020801E30BD0B56BB66B44
:100D20005ADCF90E4B6F000E4C6F97DD54DCAECFE2
:100D300060F08B800B0E0B6E260E0C6E5D0E0D6E32
:100D400001010D2EFDD70C2EFBD70B2EF9D700007D
:100D50000000200E526F170E536F000E546FC1EC3F
:100D600001F0030E0B6E080E0C6E770E0D6E0D2E3D
:100D7000FED70C2EFCD70B2EFAD75C6A5D6A800E6C
:100D800001014B6F0F0E4C6F010E4D6F16DD020E01
:100D90000C6E4B0E0D6E0D2EFED70C2EFCD7800E5A
:100DA0004B6F0F0E4C6F010E4D6F330E4E6F1BDCF1
:100DB000020E0C6E4B0E0D6E0D2EFED70C2EFCD7B8
:100DC000800E4B6F0F0E4C6F010E4D6FB9DD00C0E2
:100DD00060F0020E0C6E4B0E0D6E0D2EFED70C2E1B
:100DE000FCD7030E526F180E536F000E546FC1ECF8
:100DF00001F0630E0001616F000E626F61C0E1FFE0
:100E000062C0E2FFE66A60C04BF161C04CF162C0B3
:100E10004DF126DE61C04BF162C04CF11EDD7A0E51
:100E20000101526F180E536F000E546FC1EC01F0A8
:100E30000001B36BB46B800EB419006E800E005CC1
:100E400002E1060EB35D27E2800E01014B6F0F0E2B
:100E50004C6F010E4D6F74DD00C060F0020E0C6E21
:100E60004B0E0D6E0D2EFED70C2EFCD761C0E1FF90
:100E700062C0E2FFE66A60C04BF161C04CF162C043
:100E80004DF1EEDD61C04BF162C04CF1E6DC0001DA
:100E9000B34BB42BD0D7620E0101526F180E536FB3
:100EA000000E546FC1EC01F0800E01014B6F0F0E6C
:100EB0004C6F010E4D6F44DD00C060F061C0E1FF7A
:100EC00062C0E2FFE66A60C04BF161C04CF162C0F3
:100ED0004DF1C6DD61C04BF162C04CF1BEDCEBEC04
:100EE00002F05C6A5D6A5E6A5F6A8B80030E0B6E5D
:100EF000080E0C6E770E0D6E0D2EFED70C2EFCD745
:100F00000B2EFAD7192A19500308D8A0196A010123
:100F1000DF0E4B6F000E4C6F330E4D6F180E4E6F81
:100F2000000E4F6F48DD19500A0F026E02C001F02B
:100F30000136019001C01FF0000E015CD8A0DCD08A
:100F4000640E1F5CD8B0D8D00A0E046E1FC000F02B
:100F500043EC01F0300E00242A6E0A0E046E1FC00E
:100F600000F043EC01F008C000F0300E00242A6EBF
:100F70008B900B0E0B6E260E0C6E5D0E0D6E0D2EF5
:100F8000FED70C2EFCD70B2EFAD700000000E90E7E
:100F90000101526F160E536F000E546FC1EC01F039
:100FA000240E01014B6F000E4C6F57DC0A0E01013D
:100FB0004B6F000E4C6F29EC03F02ADC240E01016C
:100FC0004B6F000E4C6F7AEC03F0030E0B6E080EA5
:100FD0000C6E770E0D6E0D2EFED70C2EFCD70B2E41
:100FE000FAD7000E0001B61902E1000EB51907E1AB
:100FF000000EF81902E1000EF71901E1F2D7B56B06
:10100000B66B000EF81902E1010EF7190AE0800E26
:10101000006E800EF619005C02E1F551070801E34D
:101020003AD01F0E0101526F180E536F000E546F0D
:10103000C1EC01F0F90E01014B6F000E4C6F0DDC9D
:10104000F90E01014B6F000E4C6F1A0E4D6F000E22
:101050004E6F3CEC03F000C0EFF001C0F0F0000E6A
:10106000026E0150025C02E1005000080AE26B0EC1
:101070000101526F170E536F000E546FC1EC01F057
:1010800009D0CA0E0101526F160E536F000E546F35
:10109000C1EC01F009D0C30E0101526F170E536F5E
:1010A000000E546FC1EC01F08B80030E0B6E080E26
:1010B0000C6E770E0D6E0D2EFED70C2EFCD70B2E60
:1010C000FAD79A0E0101526F170E536F000E546F2C
:1010D000C1EC01F029C057F1AFEC00F02AC057F184
:1010E000AFEC00F0EBEC02F0F30E4B6F170E4C6F11
:1010F000000E4D6F4AEC02F01E0E01014B6F000E08
:101100004C6F29EC03F008EC04F0030E0B6E080E94
:101110000C6E770E0D6E0D2EFED70C2EFCD70B2EFF
:10112000FAD7000EB61902E1000EB51907E1000E5C
:10113000F81902E1000EF71901E1F3D7B56BB66BB0
:10114000000EF81902E1010EF7190AE0800E006E98
:10115000800EF619005C02E1F551040801E39ED00F
:10116000F90EEF6F000EF06FEFC0E9FFF0C0EAFF7D
:10117000EE504C0A64E1010EEF25E96E000EF021FD
:10118000EA6EEE50450A5BE1020EEF25E96E000EB5
:10119000F021EA6EEE50440A52E1040EEF25E96EAA
:1011A000000EF021EA6EEE503D0A49E1030EEF25F4
:1011B000E96E000EF021EA6EEECF1FF036D000018E
:1011C000050EEF25E96E000EF021EA6EEE50310AB1
:1011D000D8B48998050EEF25E96E000EF021EA6E6D
:1011E000EE50300AD8B4898827D00001050EEF25CB
:1011F000E96E000EF021EA6EEE50310AD8B48996FD
:10120000050EEF25E96E000EF021EA6EEE50300A71
:10121000D8B4898611D0E30E0101526F170E536FB7
:10122000000E546FC1EC01F007D01F50520AC7E006
:101230001F50560ADAE0EFD70001EF6BF06BF90EA2
:1012400001014B6F000E4C6F4F0E4D6F000E4E6F35
:101250003CEC03F000C0EFF001C0F0F0000E026EB5
:101260000150025C02E10050000818E20101196B14
:10127000130E526F180E536F000E546FC1EC01F035
:10128000FD0E01014B6F000E4C6F2DEC04F0EBECEA
:1012900002F0EFC0E1FFF0C0E2FFE66A000E0001DD
:1012A000F81902E1020EF7190CE1050E0101526F67
:1012B000170E536F000E546FC1EC01F00001F76B75
:1012C000F86B800E01014B6F0F0E4C6F010E4D6FCE
:1012D000DDEC03F0800E4B6F0F0E4C6F010E4D6F67
:1012E000CC0E4E6FF3EC02F0800E4B6F0F0E4C6F76
:1012F000010E4D6F440E4E6FF3EC02F0020E0C6EB9
:101300004B0E0D6E0D2EFED70C2EFCD7800E4B6FA4
:101310000F0E4C6F010E4D6FDDEC03F0800E4B6F26
:101320000F0E4C6F010E4D6FCC0E4E6FF3EC02F0B2
:10133000800E4B6F0F0E4C6F010E4D6FBE0E4E6F39
:10134000F3EC02F0800E4B6F0F0E4C6F010E4D6FE1
:10135000A0EC04F000C0F1F0000E0001F26F800E6E
:1013600001014B6F0F0E4C6F010E4D6FA0EC04F09E
:1013700000C002F0016A01500001F1270250F2237F
:10138000800E01014B6F0F0E4C6F010E4D6FA0ECE4
:1013900004F000C01FF0800E4B6F0F0E4C6F010E5B
:1013A0004D6FA0EC04F000C01FF0630E0001616FF0
:1013B000000E626F61C0E1FF62C0E2FF430EE66EA5
:1013C000010E6125E16E000E6221E26E480EE66EAE
:1013D000020E6125E16E000E6221E26E29C0E6FF79
:1013E000030E6125E16E000E6221E26E2AC0E6FF67
:1013F0005CC04BF15DC04CF1040E612501014D6FE5
:10140000000E0001622101014E6F94EC03F061C0F7
:101410004BF162C04CF17AEC03F061C04BF162C059
:101420004CF12DEC04F0470E01014B6F180E4C6F80
:10143000000E4D6F4AEC02F0F1C04BF1F2C04CF1DE
:1014400067EC02F000C01FF061C04BF162C04CF1CC
:101450007AEC03F03FEC04F0500E0101526F180ECD
:10146000536F000E546FC1EC01F061C04BF162C0CC
:101470004CF12DEC04F0EBEC02F0140E4B6F000E6F
:101480004C6F29EC03F0000EB61902E1000EB519FD
:1014900001E1F9D708EC04F05C4A5D2A33D5FFD7A7
:10188A0010EE24F00A0E006E010E016E3D0EF66E89
:10189A00180EF76E000EF86E98EC04F010EE19F0C0
:1018AA00010E006E010E016E060EF66E000EF76E48
:1018BA00000EF86E98EC04F010EE2EF0210E006E79
:1018CA00010E016EA90EF66E160EF76E000EF86E78
:1018DA0098EC04F010EE1AF0030E006E010E016E81
:1018EA00860EF66E180EF76E000EF86E98EC04F07F
:1018FA0010EE4FF0050E006E010E016E810EF66EAF
:0E190A00180EF76E000EF86E98EC04F0120046
:0100060000F9
:1014A000204469726563746F72793A20433A5C5FD5
:1014B0004D696B726F435C5F4D657350726F6A6507
:1014C00074735F4D696B726F435C5F484331325F89
:1014D0005472616E736365697665725F3433334D40
:0514E000687A0D0A000E
:1014E50020464F534320696E7465726E6520203126
:1014F500364D487A20766961205031384632364B70
:1015050032325F464F53435F696E7465726E655F35
:0F15150031364D687A2E6366677363680D0A007E
:101524000D0A204C65637475726520536574746983
:101534006E6720204843313220636F6E63656E749A
:1015440072617465757220737572204261736520CF
:071554005049430D0A20007D
:10155B0020506F727420486172642055415254318F
:10156B002031393230302C4E2C382C31202852433C
:10157B00363D5458205243373D525829200D0A000E
:10158B0020536F75726365205031384632364B32BB
:10159B00325F436F6E63656E747261746575725FF3
:1015AB00484331325F3139303930342E630D0A0004
:1015BB0020436F6E666967203A20503138463236C9
:1015CB004B32325F464F53435F696E7465726E6583
:1015DB005F31364D687A2E6366677363680D0A0058
:1015EB002050726F6A6574203A205031384632367B
:1015FB004B32325F436F6E63656E747261746575E7
:0F160B00725F484331322E6D637070690D0A00B3
:10161A002041766563205458205541525433204165
:10162A00534D2073757220524132206F7574707554
:04163A00740D0A0021
:10163E00205241303D41444320205241313D4F57CD
:10164E00532073656E736F722044533138423230BB
:04165E00200D0A0051
:10166200204D435520203A31384632364B32322013
:10167200416C696D2E203D2020332E3620E020352E
:04168200560D0A00F7
:1016860020496E69742053657474696E672020431F
:10169600616E616C203130206D6F64652020465587
:0316A600332000EE
:1016A900A01400EB1500621600BB1500E514005BE1
:1016B90015003E16008B15001A16008317005317E4
:0116C9000020
:1016CA0020504220737572204368616E67656D65AC
:0F16DA006E742064652043616E616C200D0A0000
:1016E9000D0A456E766F6920436465205365742041
:0C16F9006368616E6E656C203A20200072
:10170500205042206465626F7264656D656E742059
:0B17150062756666657231200D0A00E7
:1017200020546573742072656769737472657320E1
:0A173000445331384232300D0A00F4
:10173A002049542055415254312052433620262004
:09174A0054696D6572310A0D004D
:10175300204C616E67616765204D696B726F432032
:08176300372E3530200D0A007D
:10176B00204368616E67656D656E742043616E61C1
:08177B006C204F4B200D0A0009
:1017830020454550524F4D206E6F6E207574696C25
:071793006973E9650D0A000E
:10179A00E0206C2765636F7574652064752043418A
:0517AA004E414C20003F
:1017AF0020496E69742049324331203430304B6800
:0417BF007A0D0A0095
:1017C300204E4F20726573706F6E7365200D0A0093
:1017D3003031323334353637383941424344454664
:1017E3004E6F20636F6D7072656E646F200D0A001B
:1017F30057616974696E67206D736720210D0A0054
:101803002046616D696C7920436F6465203A20003E
:0C1813004D7367207265E775203A2000D5
:0A181F00205265746F75723A2000C4
:0A18290041542B433031300D0A000A
:0A18330041542B433030300D0A0001
:0A183D0041542B433031300D0A00F6
:091847002020445323313D200010
:091850002020445323313D200007
:0918590041542B4655330D0A00E1
:0818620020204352433D200009
:08186A0041542B52580D0A00F5
:0818720041542B52580D0A00ED
:07187A00204944313D20002C
:051881004D73673D00FE
:031886004F4B00C5
:020000040030CA
:0D000100281F3CFFBF81FF0FC00FE00F4024
:00000001FF
